:10014000021D800A0A5052494E540D0A80140A506A
:1001500052494E540D0A801E205052494E542022BE
:10016000544154544C4554414C45204D4F44454C0A
:100170002023223B0D208028105052494E54204D00
:100180004F44454C0D1080320A5052494E540D0ACE
:10019000803C225052494E5420222020532F4E2082
:1001A000222C20534E25313030303030303030303A
:1001B0000D2280462A5052494E542022284329209D
:1001C00031393839204F4E53455420434F4D505507
:1001D00054455220434F52502E220D2A80500A502F
:1001E00052494E540D0A805A2F5052494E542022E3
:1001F0005454424153494320222C564552532F31E7
:1002000030302C222E222C2330322C5645525325AE
:0D0210003130300D2F8064084E45570D0829
:10C000008E00FFBDF6DC8621BDFBA3BDC0C842C0CB
:10C010002743C03044C03946C07B4DC12B50C29F1E
:10C0200052C27653C0AA00BDFBA3717F147EFBFAF7
:10C03000BDFBA3BDF6DC7EC706BDC0E33CBDFD3E37
:10C04000BDFBC8383CC610A600BDFD43BDFBCC08F7
:10C050005A26F4BDFBC838C610A60081202C0286E3
:10C060002E817F2F02862EBDFBA3085A26EBBDF63C
:10C07000DCBDC128812E26C47EC000BDFBA3BDFB54
:10C08000CCBDC0F6183C862CBDFBA3BDC0F6DD566A
:10C09000862CBDFBA3BDC0F637BDF6DC3238A70049
:10C0A000089C5626F9A7007EC000BDC0E3BDFD3E3A
:10C0B000BDFBC8A6009753BDFD43BDFBC8BDC0F680
:10C0C000E700BDF6DC0820E5383CBDC128A100270B
:10C0D000096D0027F308080820F3333336EC011804
:10C0E000326E00BDFBA3BDFBCC7F00527F0053BD71
:10C0F000C0F6187EF6DCBDC128812E26037EC00066
:10C10000810D2603DC5239803025EB810A25088019
:10C110000725E3811024DF9746BDFD4BDC52050562
:10C120000505DB46DD5220CE7EFB66BDFBA3BDF6DA
:10C13000DCBDFB3126FB71F8175FF740005CC120C6
:10C1400027057C001720F371F8175FF140002738AE
:10C15000B64000363771F817CEC1754FBDF55D3268
:10C160008A30BDFBA3CEC17D4FBDF55D328A30BDA7
:10C17000FBA37EC0003A2042414E4B200020524596
:10C1800041445320415320005CC12027057C001707
:10C1900020B971F817CE4002EF001805847F8B405C
:10C1A000188C400026F2CE4002AC002743DF46EE5A
:10C1B00000DF4871F817BDF6DCCEC1E14FBDF55D7B
:10C1C0009648BDFD439649BDFD43CEC1E64FBDF542
:10C1D0005D9646BDFD439647BDFD4371F8177EC091
:10C1E0000053454520002041542041444452200042
:10C1F0001805847F8B40188C400026AD8601974639
:10C2000071F81796179A469717CE40004F5FED00CA
:10C21000EC00261E4353ED00A300261F08088CC027
:10C220000026EB7C00469646812026D771F8177EC3
:10C23000C000CC0000ED00EC002007CCFFFFED00BB
:10C24000EC003C373671F817BDF6DCCEC26B4FBD43
:10C25000F55D323318BDFD3E8640BDFBA3383CBDC5
:10C26000FD3E38EC004353ED0020F8424954204590
:10C2700052524F522000BDFBA3BDF6DC4F36323682
:10C28000BDF75CDE56BDFD3EBDFBC8324C3681407D
:10C290002709840726E8BDF6DC20E3327EC000BD16
:10C2A000FBA3BDF6DC7F0053BDC0F6C43F37BDFB2A
:0DC2B000C8BDC0F6DD5632BDF7A67EC00049
:10C4000000000030303030303030303030300D54BB
:10C410004154544C4554414C45204D4F44454C20CB
:10C420003220202843292031393839204F4E5345B6
:10C430005420434F4D505554455220434F52502E97
:10C440000D4C495354CB34545952554ECAD25052C4
:10C45000452A52554ECACB462452454D494E44CFEB
:10C46000B3465245D76F414F4E454F4ED8124141CA
:10C4700041454F4646D80D42424E455854C9505446
:10C480004F4C4554CE975641524946CDDB4E4F5402
:10C4900045474F544FCB1C454E474F535542CD86D1
:10C4A0005352455455524ECDAF464F52C8C84745DA
:10C4B000544255525354CEA75853544F5245CEED83
:10C4C0004150534554D3AE564150434C52D41C5462
:10C4D0004553444FDAE631313143414C4CDC1132A3
:10C4E00032434F554E54DD6F45534C454550D33084
:10C4F000525550524F47DBA95855474554D50D4426
:10C5000046544F4E45D78A52535553454E44D484D2
:10C510002F4F4E455252D66B2352415445DD48545D
:10C520005941534DDFD34A4E4B52454DCDCC41522C
:10C530004B5052494E54CC6553584D4954D83A57F4
:10C540004F53544F50CAC5544F4954455854D68B35
:10C550004F4F54455854D727475354494D45D85702
:10C56000405254494D45D9AD4041444C4F4F50DEA7
:10C57000D55653544F5245DC9456474554DCCE3380
:10C5800033494E505554CE0038585348414B45D846
:10C590001D4F46464C44D16C454F4E4C4F4144DDF7
:10C5A000AD44494DDD005245414E4557CAB14F4C4F
:10C5B00044434F4EDD22444545CE91544FC8EB468F
:10C5C000524F4DF3BF53544550C9004154C906431F
:10C5D00048414EE6955459474554E6C326474F50C7
:10C5E000494EE741544845534449EA9B2020205096
:10C5F0004552494F44EB82414253E6804245455300
:10C600005152E7C647415454454D50E8604849539C
:10C61000494EE9244F46464153494EE9904E554311
:10C620004F554E54EAEE454C4F47EC3A494E47457C
:10C630005850EDF549524556455253EA845A5953DC
:10C640004EEA9050495A454D4F44454CEA7B53E6DB
:10C650004C3DE4D2252F2F2A343E3DE4A32F233C2A
:10C660002F3E3CE4AE7E2F2A3C3C3EE4AE2B3D2DDB
:10C670003E3EE4C0454E442E2E3C3DE4C93F2F3E95
:10C680003E3CE4D93C3E3C0404E4E08EBFFF7F0026
:10C69000760E86FF9791BDFB04861A97111A1ABD74
:10C6A000FB044FCE738C6F00088C73A226F87F00BA
:10C6B000B37F00B4CC0C00FD72887F00B57F006AA8
:10C6C0007F0076860AB7B59ACC1770DDAF863997AA
:10C6D0009F9797979497A597A897A2867E97ABCC9C
:10C6E000FBA3DDACCC0000DD9ADD9C7F0077BDF6BE
:10C6F000DC86FF978C979E7F00927F00B67F009329
:10C700007EC84B4F4B0D8EBFFF86FF979E860AB7A4
:10C71000B59A7F00817F008CBDF6DCCEC7034FBD8C
:10C72000F55DCEC729FF738CCE0000FF7394FF73B5
:10C730008E863EBDFBA34FCEB294BDF46D083CCEB9
:10C74000B294865CBDEEFB261EBDE41EFC721893FF
:10C75000522607FC721A935427033820D4865CBDF6
:10C76000EEFB27037EF3BF1838DF5618BDEF80DCE1
:10C7700056DD4EBDEF0BDC522634DC54261B8627DB
:10C78000BDEEFB27AC7EC87A45444954494E47204C
:10C7900044495341424C45440D7D0092270DCEC77C
:10C7A000884FBDF55DBDF6DC7EC7314D2A06CC0055
:10C7B000087EF01F0909098A80ED00DF46DC4E93F0
:10C7C00046E702DE4E09E700FE73A209FC73A2E011
:10C7D00000820018EC00847F9354FE73A22505BDEF
:10C7E000F4DA2705FF73AE201BFF73A6FF73AEFCC0
:10C7F00073A2FD73A8BDF4FEFF73A4BDF64EFC73D7
:10C80000A6FD73A2DC4E9346C10526037EC731FE0A
:10C8100073A2FF73AAF373AAFD73AC188CB28F18BE
:10C8200023037EF464FD73A2BDF667FC73AEFD7353
:10C83000A6DC4EFD73A8DC46FD73A4BDF64E7EC794
:10C8400031CE01006F000926F8203AFEB5CD8C30BC
:10C85000392722B6C42E815326E7CE0142FF73A4A6
:10C86000CE73D2FF73A6FC0140FD73A8BDF64EFC4B
:10C8700073A6FD73A27ECACE0000CCC878FD738C6F
:10C88000CCC441DD520908A600B1C42B27F8DF460D
:10C89000A6003CDE52E6002B2811270B18C3000827
:10C8A00018DF5220F0DE4A08E600DF4A38083CE193
:10C8B0000027F2C180240838DE463CDE5220DDDE4F
:10C8C0004A08A60038363739BDF6A7BDF377DC52E3
:10C8D000FD7394B6C42C814F2709FC739483000424
:10C8E000FD7394CCC5BBDD527EC885BDE41EDC540F
:10C8F000FD7398DC52FD7396CCC5C5DD527EC885AC
:10C90000BDE41E7EC90FCC0001DD545F4FDD52DC5B
:10C9100052FD739ADC54FD739CFC738CFD739EFF77
:10C9200073A030200518C3000E18EC00271C18BC9B
:10C9300073941826F0FF73AA18C3000EFD73AC3071
:10C94000FF73AEBDF667FE73AC35FE73A07EEF12CB
:10C95000BDEF1824037EF3BFFD73903CFE73942655
:10C9600004387EF3BFBC7390270738BDF6807EC9BC
:10C970005BEC02F3739CED02EC00F9739BB9739AC4
:10C98000295BED00FC739A2B267D73962A066D00B9
:10C990002A4D20046D002B39EC0018BC739625310C
:10C9A000263D18EC0218BC73982526272420307DDC
:10C9B00073962B066D002B2720046D002A13EC00C4
:10C9C00018BC73962519260918EC0218BC73982513
:10C9D0000E38FC739EFD738CFE73A02006ED0038AC
:10C9E000BDF6807EEF12BDE41EDC522605DC544D00
:10C9F0002A09CC00087EF01F7EF3BF3637862CBD97
:10CA0000EEFB26F4BDE41EDC5226E7DC544D2BE29F
:10CA10003332DD48DC54934825D83CFE738CEC005F
:10CA2000847FDD502733189C48252E9C54270224F0
:10CA300028BDF6DCCECA3F4FBDF55D387EC7064344
:10CA4000414E4E4F5420455241534520435552527A
:10CA5000454E54204C494E450DDE54DF52DE48DF32
:10CA600054CE73D2BDF4EC2404387EEF12FF73A6CB
:10CA7000DC52C30001DD54BDF4EC2408FC73A6FDB8
:10CA800073A22012FF73A4FE73A2FF73A8BDF64E1B
:10CA9000FE73A6FF73A2DE5027CFDF54CE73D2BD44
:10CAA000F4EC080808A600810D27BF813A27BB20B7
:10CAB000F3BDEF0B810D2707813A27037EC9E6CC32
:10CAC00073D2FD73A2BDF3B47EC706BDF3B486FF77
:10CAD0002004BDF3B44F978C7F0081CE73D27F00CA
:10CAE000547F0055BDF4EC24037EC706FF738C967B
:10CAF000B5271BBDFBA3EC00847FDD547F00527F74
:10CB0000005386019745BDF598863EBDFBA30808F6
:10CB100008BDF6EDCCC479DD527EC885BDE41E3C6F
:10CB2000BDF3B4BDF511270738CC00157EF01F32D8
:10CB3000327ECAECBDEF1824037ECBD13CFD73AA34
:10CB400018EC00DD64EC02DD66CCF0E9DDAC387F8A
:10CB500000547F0055862CBDEEFB260DBDEF80DC1A
:10CB6000522706CC00087EF01FDC542BF636379691
:10CB7000442729862CBDEEFB270A862DB1C42EBD85
:10CB8000EEFB2613BDEF8096442711DC5226D4DC41
:10CB9000542BD0DD5E200ACC00002003CC7FFFDDCB
:10CBA0005E3332DD543CBDF4DA2512BDF629BDF406
:10CBB000EC250AEC00847F935E27F025EEFE73AA35
:10CBC000DC64ED00DC66ED02CCFBA3DDAC387EC797
:10CBD00006BDEF80DC522706CC00087EF01FDC5437
:10CBE0002BF6363796442729862CBDEEFB270A867E
:10CBF0002DB1C42EBDEEFB2613BDEF809644271148
:10CC0000DC5226D4DC542BD0DD5E200ACC00002080
:10CC100003CC7FFFDD5E3332DD5496763686019796
:10CC2000763CBDF4DA2517BDF6297D0093262ABD92
:10CC3000F4EC250AEC00847F935E27EB25E938327B
:10CC400084019776863BBDEEFB260BBDFB66811308
:10CC500027F9811127F57EC706383284019776BD02
:10CC6000FB047EC706863BBDEEFB26037EEF1286E5
:10CC70000DBDEEFB270C863ABDEEFB27058D0A7E27
:10CC8000EF1209BDF6DC7EEF1286019745BDF57106
:10CC900027698623BDEEFB2639C600A60081302613
:10CCA00002C680D745BDE41E9655847F9A459745B8
:10CCB0008648C610A10027138642C602A100270B92
:10CCC0008651C608A1002703C60A0908F7B59A7E4F
:10CCD000CCFBA600815C260A08BDE41E96559DABE0
:10CCE0002019867BBDEEFB260CBDCD20867DBDEEDA
:10CCF000FB26252006BDE41EBDF598862CBDEEFB67
:10CD0000278B863BBDEEFB260139860DBDEEFB274A
:10CD10000A863ABDEEFB27037EF3BFBDF6DC093978
:10CD2000BDE41EBDCF8CDC523637DC543637862C42
:10CD3000BDEEFB26E3BDE41EBDCF8C3332DD4833B0
:10CD400032DD469352250E2706CC00167EF01FDCFE
:10CD500054934825F4BDCD6FBDF144BDCD6F9DAB5F
:10CD6000DC46935225EF2606DC54934824E7393CF1
:10CD7000DE463CDE483CDE64DF46DE66DF4838DF08
:10CD80006638DF643839BDF6A7BDE41EBDF3B43C98
:10CD9000BDF511270738CC00157EF01F18FE738CE7
:10CDA0003CFE738E3C7F7394BF738E187ECAECBDBD
:10CDB000F3B4FC738E26037EF3BFBE738E38FF730D
:10CDC0008E38FF738C38BDF6807EEF12FE738C7F39
:10CDD00000547F0055BDF4FE7ECAE7BDE41EDC5260
:10CDE0002604DC5427037ECB11BDF50825037ECA3B
:10CDF000EC7EC706BE739238FF738C3838BDF6DC04
:10CE00003CBDF5712609BDEF18DD54256820233C93
:10CE1000BDEF18DD5424037EF3BFA600B1C42D97E7
:10CE2000454FA70038BDF55D964509A700863ABD78
:10CE3000FBA33CFE738C3CCEFFFFFF738CBF739251
:10CE4000DC543736863ACEB394BDF46DCEB394A697
:10CE500000810D2606A7018630A700BDE41EBDEFA8
:10CE60000B810D268F380FDC54ED02DC52ED000EE5
:10CE700038FF738C3832B1C43132863BBDEEFB27AC
:10CE800003BDF6DC862CBDEEFB26037ECE007EEFD6
:10CE900012A600810D270ABDF377862CBDEEFB2775
:10CEA000F67EEF127EF3BFBDCF73862CBDEEFB2660
:10CEB000F3BDE41E3CDE522609DE5427058C000932
:10CEC000250738CC000B7EF01F183837C601D75223
:10CED000862CBDEEFB260DA600803025C7810324DD
:10CEE000C3975208323CD652BDF99F202CBDCF7358
:10CEF00086319762862CBDEEFB261D8623BDEEFB98
:10CF00002631A600088132270B813427078131277B
:10CF1000037EF3BF976220DC3CFE73AAB6C42D816A
:10CF20004E2704DC422002DC66ED02DC64ED0038B2
:10CF30007EEF12BDEF0B8127270481222610CCF053
:10CF4000E9DDACBDCC89CCFBA3DDAC7ECF18BDE464
:10CF50001ED662C134260C9652BDF0E99653BDF040
:10CF6000E92004C13226059654BDF0E99655BDF07E
:10CF7000E92081BDEF182511FD73AA3CFE73AAECD0
:10CF800000DD64EC02DD6638397EF3BFCC000FDDD6
:10CF900046CC8000D39CDD48DC46D99B999A9352BD
:10CFA000250B2608DC4893542503270139CC0016AD
:10CFB0007EF01F3CFC73A28373D22604387EEF12EE
:10CFC000188C3EBF2522CECFD04FBDF55D7EC70663
:10CFD00050524F4752414D20544F4F204249472015
:10CFE000464F5220524F4D0018C30142FD73D0CE20
:10CFF000D3034FBDF55DBDF6DCCE177096431A9195
:10D000004327FBBDFB2C260D0926F1CED3134FBDC4
:10D01000F55D7EC706BDFB66811826037EC70681C7
:10D020001526D9CEB601DF5286019755FC73A2DDD5
:10D030004ACC8D70DD4CCE73D0BDD07638862BBDFA
:10D04000EEFB3C260C4F5FDD4CDD4ACEC000BDD070
:10D05000764FCED061A60081242714BDD0F80820D9
:10D06000F43A303030303030303030300D0A24BDBA
:10D07000D149387EEF12DF4E7F00467C0046089C87
:10D080004A27069646811026F2863ABDD0F87F00E0
:10D09000479646BDD0D7DC4ED34C37BDD0D732BD36
:10D0A000D0D74FBDD0D7DE4EA600BDD0D7089C4A02
:10D0B00027107A004626F14F9047BDD0D7BDD0CC7F
:10D0C00020B44F9047BDD0D7BDD0CC39860DBDD050
:10D0D000F8860ABDD0F839369B47DD4732364444DE
:10D0E0004444BDD0EA32BDD0EA39840F8B30813A56
:10D0F00025028B07BDD0F8393CDE52A7008CB680E4
:10D10000270608DF5238393CCEB601DF524F97541C
:10D110008601BDFBA39655BDFBA343BDFBA3A600A3
:10D12000BDFBA39B549754088CB68126F19654BD41
:10D13000FBA3BDFB66811527CF8106270781182633
:10D14000C77EC7067C00553839DE528CB681270B66
:10D150006F00088CB68126F8BDD1078604BDFBA3FD
:10D16000BDFB66811827DA810626DE39BDE41EBDC7
:10D17000CF8CDC52DD64DC54DD66862CBDEEFB27F3
:10D18000037EF3BFBDE41EBDCF8CBDD2F82406CC18
:10D1900000167EF01FB6C42E81532708DC529A4039
:10D1A000DA41DD5218DE523CDE543C18862CBDEECE
:10D1B000FB2707CC177036372020BDE41EDC522732
:10D1C00006CC00177EF01FDC543637862CBDEEFBF4
:10D1D0002608BDEF1824067EF3BFCC004EDD4E338B
:10D1E00032DD501838DF5438DF52183CDE4E8C00E8
:10D1F0004E260ACED3034FBDF55DBDF6DCBDD2167B
:10D200002626DE4E8C004E260ACED3134FBDF55D8A
:10D21000BDF6DC7ED2EADE5096431A914327FBBD71
:10D22000FB2C26030926F139BDFB66811826037EF7
:10D23000D2EA811526C78601974720347C0047BD76
:10D24000D216260D3338BDD2F824037ED2CA7ED240
:10D25000EABDFB66333881062716811826037ED285
:10D26000EA811527043C3720D6DF66D7657A004768
:10D27000BDD2F8254BDE663CD665377F005A7F006D
:10D280005B8601BDFBA39647BDFBA343BDFBA3BDCE
:10D29000D2F82515965A8180271EBDF144BDFBA307
:10D2A0009B5B975B7C005A20E6965A818027094F4A
:10D2B000BDFBA37C005A20F1965BBDFBA37ED23C54
:10D2C0008604BDFBA3BDD2162619730064730065E6
:10D2D000DC664353C30001DD66DC64C9008900DD00
:10D2E000642007BDFB66810626D6DE4EDC64ED00B9
:10D2F000DC66ED02387EEF12965390652604DC540E
:10D3000093663957414954494E4720464F52204E63
:10D31000414B004E414B204E4F5420464F554E44FA
:10D32000204245464F52452054494D454F555400E3
:10D33000BDE41EDC522706CC00187EF01FDC54260C
:10D340000D96431A914327FB4FDD6C7EEF12DD6E85
:10D35000200108A600B1C43127F8813A272C810D9D
:10D3600027283C20091ADC6C936E270B24097B408C
:10D370001520F2387ECB11DD6C38CC0000DD54BDB9
:10D38000F50825037ECAEC7EC7063C1ADC6E936C5A
:10D39000270925022AF5862ABDFBA3CE0000DF6CF3
:10D3A000387EEF129DA53838CC000C7EF01FBDE40E
:10D3B0001EDC52270DCC000C7EF01F3C8DE6387E23
:10D3C000EF12DC544D26F4C10225F0C10E24ECC14D
:10D3D00008241786805D2704445A20F9369A159749
:10D3E00015329A8B9720978B201EC00886805D2768
:10D3F00004445A20F9B1C43124024444369A0397B4
:10D4000003329A8A9701978A862CBDEEFB279F7E6E
:10D41000EF129DA83838CC000C7EF01FBDE41EDC56
:10D4200052270DCC000C7EF01F3C8DE6387EEF12AB
:10D43000DC544D26F4C10225F0C10E24ECC10824B1
:10D440001886805D2704445A20F9364394159715B1
:10D45000329A8B9720978B2021C00886805D270405
:10D46000445A20F9B1C4312402444436439403970A
:10D4700003329A8A9701978AC00E862CBDEEFB274D
:10D480009B7EEF12BDD5FD86809A8A9701978ABD53
:10D49000EF0B8122270481272610CCD4E0DDACBD20
:10D4A000CC89CCFBA3DDAC7EEF12BDD645DC7B2660
:10D4B00004DC79271BBDF144BDD4E0DC7B83000193
:10D4C000DD7BDC79C2008200DD7926E9DC7B26E5A4
:10D4D0003CFE73AADC64ED00DC66ED02387EEF12E0
:10D4E0003CDE7D8C011324010FBDD5F7717F03BD98
:10D4F000D5F7C608442505717F03200572800320F7
:10D5000000BDD5F75A26ED728003380E39BDD5FD22
:10D51000BDD645862CBDEEFB27037EF3BFBDE41EC2
:10D52000DC7B2607DC7926037ED4D086FE948B979D
:10D5300020978B867EB7010CCCD59EFD010DDC5269
:10D540002706CC00257EF01F0FDC42D354DD54DCCF
:10D5500040D9539952DD5296AE8900974E7F007F95
:10D56000DF467F0080DC7D83011325037A00800E77
:10D5700001010F7201140E1A0F967F2616964E9017
:10D58000AE251026EADC529340250826E2DC5493AF
:10D590004224DC71FE140E86FF97807ED4D071FE8B
:10D5A00014968027010ED61737C4F7D717DC7D04F1
:10D5B000D37D18BDD5F9C68096150425070101BD98
:10D5C000D5F720F417DE46BDF0E9DC7B830001DDF2
:10D5D0007BDC79C2008200DD79DC7D04047B0115EF
:10D5E000260583000126F6DC792608DC7B260486E6
:10D5F000FF977F33D7173BDE7D0926FD39BDE41E3B
:10D600003CDC52DD46DC54DD48BDF09ECC04B07BF2
:10D6100001BB2703CC0960DD53BDF17FDC52260C32
:10D62000DE548C0FA024058C001E240A38CC00196F
:10D630007EF01F7EF3BF18830007DD7D38862CBD8A
:10D64000EEFB26EF39BDE41EDC52DD79DC54DD7BD8
:10D65000862CBDEEFB26DCBDEF1825D7FD73AA3C5A
:10D6600018EC00DD64EC02DD663839BDE41EBDF364
:10D67000B43CBDF511270A387F0081CC00157EF03F
:10D680001FDF823886FF97817EEF12BDCF73860D34
:10D69000B773AC862CBDEEFB2616865CBDEEFB2672
:10D6A00036BDE41E9655B773AC862CBDEEFB27271E
:10D6B0003C4FCEB394F673ACBDF46FCEB394A600DA
:10D6C000B173AC270C08DF5238BDF0E93CDE5220C4
:10D6D000EDBDF0E97ECF19BDE41EDC522706CC007B
:10D6E0001A7EF01FDC542732DC54DD52BDFB2C27A0
:10D6F0000FBDFB6636BDF0E932B173AC271920E8E7
:10D7000096431A36BDFB2C3226E7914327F4DC52B0
:10D71000830001DD5226E97ECF18BDFB2C27F8BD22
:10D72000FB66BDF0E920F0BDCF73860DB773AC8604
:10D730002CBDEEFB2612865CBDEEFB27037EF3BFFD
:10D74000BDE41E9655B773AC3CBDF144B173AC2734
:10D7500005BDF6DE20F33836863BBDEEFB32270CE6
:10D76000810D2605BDF6DC2003BDFBA37ECF18BDD1
:10D77000F3B4CCB28FB373A2DD547F00527F005359
:10D7800086069745BDF5987EC706BDE41EDC522788
:10D7900006CC001B7EF01FDC54188C00DC1825F131
:10D7A0003637862CBDEEFB26E8BDE41EDC5226E1B2
:10D7B000DC5426043232203505DD5425D43332DDE5
:10D7C000463C867EB70106CCD7F0FD010771FD030C
:10D7D0009608DC09D346DD0B8601970F860897086B
:10D7E0001ADC4626FB7F00088600970F387EEF1272
:10D7F0009608DE54270E09DF5488019708DC0BD306
:10D8000046DD0B3BDC0BD346DD0BDF463B86FF36AC
:10D8100020024F36BDF3B43297927EC706BDE41E98
:10D82000DC522706CC001C7EF01FDC542706DDAF3F
:10D83000860120014F97767EEF12A600812D260DDE
:10D84000BDFB3126FB86FF0897777EEF12812B27E1
:10D85000037EF3BF4F20F0B673B0BA73B1BA73B49E
:10D86000BA73B5BA73B8BA73B9BA73BCBA73BDBA7E
:10D8700073BEF673BF271FC12025028AFFBA73C08B
:10D88000BA73C1BA73C2F673C3270BBA73C4BA733F
:10D89000C5BA73BE2706CC00267EF01F7F004A7FE4
:10D8A000004BFC73B2DD4CCC003CDD484F5FDD46E5
:10D8B000DD52FC73B6DD54BDF2B3BDD9924F5FDDCE
:10D8C00046DD52CC0E10DD54FC73BADD48BDF2B318
:10D8D000BDD9924F5FDD465CDD52F673BF5ADD481D
:10D8E000CC5180DD54F673C7C1292404CB14200821
:10D8F000C0502515C1142411D75E54545C4FD34831
:10D90000DD48F673C3C10D2506CC001D7EF01FD780
:10D91000463CCED9A1C1032409D65EC40326037AAE
:10D9200000495F7A00462707EB0089000820F43899
:10D93000D348DD48BDF2B3BDD9924F5FDD52D65E0C
:10D94000DD54CC01E1DD46CC3380DD48BDF2B3BD12
:10D95000D992BDEF18250E3C18DC4AED00DC4CEDE9
:10D9600002387EEF12DC4CDD484FD64BDD465FDDE2
:10D9700052C664DD54BDF2B30FDC50DD42D64FD742
:10D98000418664D64A3DDB4E8900D74097AE0E7E75
:10D99000EF12DC50D34CDD4CDC4ED94B994ADD4ABA
:10D9A000391F1C1F1E1F1E1F1F1E1F1E1FBDEF180D
:10D9B0003C24460F96AE9752DC40DD53DC4297552F
:10D9C0000ED75ECC0064DD485FDD46BDF17FDC53E1
:10D9D000DD5F965597619651D65EDD544F5FDD52FF
:10D9E000DD46C664DD48BDF17FDC549B61DD54DC5F
:10D9F0005FC9008900DD52200918EC02DD54EC00FB
:10DA0000DD52188C8000250738CC001E7EF01FCC1C
:10DA10000001DD46CC5180DD48BDF17FDE543CDCA9
:10DA20004EDD52DC50DD544F5FDD46CC0E10DD483C
:10DA3000BDF17FDC54FD73BA5FFD73B8DC4EDD527F
:10DA4000DC50DD544F5FDD46CC003CDD48BDF17F4E
:10DA5000DC54FD73B65FFD73B4DC50FD73B25FFD43
:10DA600073B038187F00527A00527C0052BDDAD66B
:10DA7000260A83016E24F3C3016E200883016D24FE
:10DA8000E9C3016D3637D652CB50C1642502C0645C
:10DA90004FFD73C65FFD73C43332CED9A17F0054EE
:10DAA0007F00537C005337E600BDDAD6260937D60F
:10DAB00053C1023326015C08D75533935424E4D371
:10DAC000544F5CFD73BED653FD73C25FFD73BCFD46
:10DAD00073C0387EEF1236965284033239CC002060
:10DAE0007EF01F7EF3BFBDEF0B8122270481272626
:10DAF00013BDDB95CCDB78DDACBDCC89CCFBA3DDE5
:10DB0000AC7EEF12BDE41E18DE523CDE543C18869B
:10DB10002CBDEEFB26CDBDE41EDC5226C09654265D
:10DB2000BCD6552750C12124B4BDDB95D746183843
:10DB3000DF5438DF5218D64686209046270F7800EB
:10DB4000557900547900537900524A20EF7B805276
:10DB50002705720403200371FB0372041571FB1582
:10DB60007800557900547900537900525A26DE72B4
:10DB7000201571DF157EEF12C608492405720403D3
:10DB8000200371FB0372041571FB155A26EC7220F9
:10DB90001571DF153986049A8A9701978A86249A27
:10DBA0008B9720978B71DB15398627BDEEFB270AF3
:10DBB0008622BDEEFB27037EF3BFBDDBE5974EBD9E
:10DBC000DBE536BDDBE51632DD46BDDBE5BDDBE57D
:10DBD000D64E270E5AD74E3CDE46A70008DF463801
:10DBE00020EB7EEF128D0A48484848368D03331BE0
:10DBF00039A600088030250C810A250B80072504F2
:10DC0000811025037EF3BF39CC00217EF01F7EF307
:10DC1000BFBDE41EDC5226F0DC54183C18862CBD37
:10DC2000EEFB26EABDEF0B81222704812726101880
:10DC30003818DDACBDCC89CCFBA3DDAC7EEF12BDCA
:10DC4000E41E18DE523CDE543C18862CBDEEFB2749
:10DC500005CC004E2005BDEF1825B3FD73AA18387A
:10DC6000DF5438DF5238DF46183CBDFB3126FBCE8F
:10DC7000DC7B3CDE463CDC54DE52393CFE73AAEDD4
:10DC800002183818ED00387EEF127EF3BF38CC0052
:10DC9000247EF01FBDEF1825F13C188C719C25EDFA
:10DCA000EC00DD56EC02DD54188372184353C300B8
:10DCB00001541736BDF7A6DC54DD56324CBDF7A62D
:10DCC000387EEF127EF3BF38CC00247EF01FBDEF0C
:10DCD0001825F13C188C719C25ED3C188372184076
:10DCE00050C30001541736BDF75CDC56DD52324C90
:10DCF000BDF75C38DC56ED02DC52ED00387EEF12E9
:10DD0000BDE66ADC522615DC54188C0014250C8CF8
:10DD10000C01240718FD72887EEF1218CC00237EB8
:10DD2000F01F7F00B37F00B4867BBDEEFB260EBDE7
:10DD3000EF18250CDDB3867DBDEEFB26037EEF12CA
:10DD40007EF3BFC6317EF01FBDE41EDC5226F4DC3C
:10DD50005427F04D26EDD7B786C05F5C90B724FB03
:10DD60005A7B01BB2601545AD71CD7637EEF127F22
:10DD70000008BDEF18251CFDB598867EB70109CCBB
:10DD8000DD96FD010AC602D708D608DC0DDC09C6FF
:10DD900012D7087EEF129608FEB598EC02C3000178
:10DDA000ED02EC00C9008900ED00DE0D3B86FF9717
:10DDB0004F860197503CCC0052FD73ACBDEF182547
:10DDC000123637862CBDEEFB26073332FD73AC20AE
:10DDD00002323338BDE41EDC52DD64DC54DD66867D
:10DDE0002CBDEEFB27037EF3BFBDEF1825F8FD73B6
:10DDF000AA3C96B636861897B6BDFB04CE0064964C
:10DE0000431A914327F9BDFB2C26EE0926F186150E
:10DE1000BDFBA37C004FD64FC11426208618BDFB46
:10DE2000A3FE73AA4FED025FED00FE73ACDC66ED5E
:10DE300002DC64ED003297B6387EEF12BDDEC127FA
:10DE4000CDBDFB6681182604C61520D581042609A0
:10DE50008606BDFBA3D64F20C88101269CBDDE6C83
:10DE600026978606BDFBA37C005020D0CEB394C677
:10DE700083BDDEB1A700085A26F7FCB394531127DF
:10DE80000139CEB3964FAB00088CB41626F8B1B466
:10DE900016270139B6B3944C915026064A91502763
:10DEA0000139CEB396A600BDF0E9088CB41626F56C
:10DEB000393CBDDEC1382704BDFB663938387EDD0C
:10DEC000F9CE01F4BDFB2C27013996431A91432763
:10DED000F90926F0393CBDF839961784CF97178495
:10DEE000BF971786FFB7719BD6BBC408FAF8F2BD7F
:10DEF000F91C1A0FCEDF0FFF01100E387EEF123023
:10DF0000CC0032A702E701CCF01FED057EDFC1B6E1
:10DF1000719B26037EDFBEF6718FC4074FC3F8F2F4
:10DF20001896BB8408AA008A02BDF933FA717FFDF6
:10DF30007196FC7196DDBCFC7191054C812024BF6B
:10DF4000168407585858C4C0DA159A1718FC7192ED
:10DF5000847FC34000189717D715DCBCED0071F81B
:10DF600017713F15FC7192C30002FD7192F6719119
:10DF7000C900F77191F1718525162608FC7192B3DD
:10DF80007186250CFC718AFD7192B67189B7719109
:10DF9000DE6C08DF6C7A00B82619DC42C30001DDB4
:10DFA00042DC40C9008900DD4096AE890097AE96FC
:10DFB000B797B8717F1BFE718227026E003BBDF8D8
:10DFC0004ACEFBD1FF011020C738CC00017EF01FE4
:10DFD0007EF3BFBDEF18240ABDEF80964427F1CC35
:10DFE0000052FD73AA3C18EC0026DEEC02FD73AC77
:10DFF00038862CBDEEFB26D87EE00F863BBDEEFBBF
:10E0000027F63CFE73AAFC73ACED02387EEF12CC0F
:10E01000E23CDD46BDEF0BDF483CDE46A1002609B1
:10E0200008DF463808A60020F0A6002B1908A60035
:10E030002AFB0808A6002604387EF3BFDF4638DE38
:10E0400048A6007EE0193C16584FC3E22618EC00A3
:10E05000186E0038A601BDE21A387EDFFB38A60133
:10E06000BDE21A38BDE41EDC5227037EF01FDC54EB
:10E070002718830001B373AC4D2606C18024EC2021
:10E080000881FF26E6C18025E217BDE21A7EDFFB8C
:10E0900038A60138E600C1412706C14226058B108B
:10E0A0000820E736BDE41EBDE1E1270C328B30BD10
:10E0B000E21ABDE1FB7EDFFB32BBC431BDE21ABD1B
:10E0C000E2067EDFFB38A6013836BDE41EDC5227AF
:10E0D000037EF01FDC544D26F837862CBDEEFB275F
:10E0E000037EF3BFBDE41EDC5226E6DC544D26E180
:10E0F000BDE1E12616DF46183332BDE21A17BDE254
:10E100001A1817BDE21ADE467EDFFBDF46183332EF
:10E110008B107EE0FA38A601387EE0A338A60138DD
:10E12000E600C1412709C14227037EF3BF8B403679
:10E13000088623BDEEFB262EBDE41E32BDE21ABDCD
:10E14000E2067EDFFB38A6013836B6C42D802BBD33
:10E15000EEFB2612BDE41E32BDE21ABDE1FB7EDFFE
:10E16000FB38A6013836BDE41EBDE1E1260C328B3A
:10E1700020BDE21ABDE2067EDFFB9654270C328BEF
:10E1800030BDE21ABDE1FB7EDFFB328B1020E238AE
:10E19000A601BDE21A38BDE41EBDE2067EDFFB38F3
:10E1A000388622BDEEFB2604167EE1B48627A10048
:10E1B000260D1608A6000811270BBDE21A20F5BD92
:10E1C000E41EBDE206862CBDEEFB27D57EDFFB38C4
:10E1D00038BDE41EBDE1FB862CBDEEFB27F37EDFE0
:10E1E000FBA600B1C42B26030820F6812C260B08C1
:10E1F000A60008815827037EF3BF39DC52260E960D
:10E2000054BDE21A200EDC522706CC00277EF01FF8
:10E21000965426F99655BDE21A393CFE73ACA70018
:10E2200008FF73AC3839E053E05DE090E0C5E115DC
:10E23000E11CE145E161E18FE19FE1CF4E4F50806C
:10E24000014C535244800441534C44800554415086
:10E2500080065450418007494E58800844455880F4
:10E2600009434C56800A534556800B434C43800C5F
:10E27000534543800D434C49800E534549800F530D
:10E280004241801043424180115441428016544221
:10E290004180175847445880184441418019534CD5
:10E2A00050801A414241801B5453588030494E538C
:10E2B000803150554C41803250554C42803344455A
:10E2C000538034545853803550534841803650530E
:10E2D0004842803750554C58803852545380394109
:10E2E0004258803A525449803B50534858803C4DE4
:10E2F000554C803D574149803E535749803F4252DB
:10E3000041812042524E81214248498122424C5350
:10E31000812342434381244243538125424E458118
:10E32000264245518127425643812842565381292E
:10E3300042504C812A424D49812B424745812C4213
:10E340004C54812D424754812E424C45812F4E45DD
:10E35000478240434F4D82434C53528244524F5266
:10E360008246415352824741534C8248524F4C821D
:10E3700049444543824A494E43824C545354824D4A
:10E38000434C52824F41494D83614F494D83624511
:10E39000494D836554494D836B4A4D50844E5355C6
:10E3A000424486834144444486C3435058868C4C3F
:10E3B000444486CC4C4453868E4C445886CE5355A8
:10E3C000428580434D5085815342438582414E446E
:10E3D000858442495485854C44418586454F528504
:10E3E0008841444385894F5241858A414444858B05
:10E3F0005354414187875354414287C753545387ED
:10E400008F4A5352878D53544487CD53545887CFE6
:10E41000425352888D4442890044578A0000BDE42B
:10E420004EF6C431A600081127FA817C270209396B
:10E43000DC543736DC523736BDE44E32339A52DA8A
:10E4400053DD5232339A54DA55DD547EE421BDE473
:10E450007EF6C42BA600081127FA81262702093967
:10E46000DC543736DC523736BDE47E32339452D436
:10E4700053DD5232339454D455DD547EE451BDE51E
:10E4800024A60008B1C43A27F809813C2504813F3D
:10E49000250139DC543736DC523736CCC651DD52D3
:10E4A0007EC885BDE4E9250B860197552008BDE4AB
:10E4B000E926F57F00557F00547F00537F005239D5
:10E4C000BDE4E927EE25EC20DFBDE4E927DA25D815
:10E4D00020E1BDE4E926DC20CFBDE4E924D520C855
:10E4E0003233DD523233DD5439DF4E381838DF50E5
:10E4F00038183C183CDE503CDE4EBDE5243233DD9E
:10E50000463233DD4896469852182A0CDE529C4615
:10E510002610DE549C481839DE469C522604DE48FC
:10E520009C541839862DBDEEFB2606BDF09E7EE577
:10E530007D862BBDEEFBBDE58E862BBDEEFB263525
:10E54000DC543736DC523736BDE58E3233DD4632A9
:10E5500033DD48DC54D348DD54DC52974ED947991B
:10E5600046DD52964E98462BD0964E98522ACACCEB
:10E5700000097EF01F862DBDEEFB270139DC5437E4
:10E5800036DC523736BDE58EBDF0867EE54BBDE606
:10E5900022862ABDEEFB2621DC523637DC54363784
:10E5A000BDE6223332DD483332DD46BDF25DDC4E5E
:10E5B000DD52DC50DD547EE591A600812F270581D8
:10E5C000252701393C087F00447D00522A067C0043
:10E5D00044BDF086DC523637DC543637964436BDBF
:10E5E000E6223297447D00522A067A0044BDF08626
:10E5F000DC52DD46DC54DD483332DD543332DD524B
:10E600003CBDF17F38183836A60081252608DE4E3D
:10E61000DF52DE50DF54321896442703BDF0867E69
:10E62000E5910908A600812027F981302504813A67
:10E6300025308128273E81262728A6018141250CE7
:10E64000815B2408CCC5CFDD527EC885BDEF18DDC7
:10E6500052251E3C0FDE52EC00DD52EC020EDD5462
:10E660003839BDEF8096442708398628BDEEFB2750
:10E67000047EF3BF08BDE41E8629BDEEFB26F239F9
:10E68000BDE66A96522A03BDF08696522B0139CC1C
:10E69000000A7EF01FBDE66ADC522706CC000B7E26
:10E6A000F01F3C8D0838DD545F4FDD5239DE548C4D
:10E6B000000B250A9D9F3838CC000B7EF01F18BD3B
:10E6C000F8443918FE73AA3CDE643CDE663C1886CA
:10E6D00028BDEEFB2629BDCF737F00527F00537FFC
:10E6E0000054862CBDEEFB26288623BDEEFB260FAC
:10E6F000A600088134270B81322711813127127E31
:10E70000F3BFBDF1449752BDF1449753BDF1449717
:10E7100054BDF14497553CFE73AADC66ED02DC64FF
:10E72000ED00381838DF6638DF6438FF73AA1886C2
:10E7300029BDEEFB26C9399DA23838CC000C7EF0ED
:10E740001F8628BDEEFB265BBDF09EDC54053736E8
:10E75000BDE41EDC52270CCC000C7EF01F3C8DD794
:10E76000382025DC544D26F5C10225F1C10E24EDDB
:10E77000C108243386805D2704445A20F936439427
:10E780008B9720978B32941527073233C3000120D3
:10E79000023233DD54862CBDEEFB27AF8629BDEE59
:10E7A000FB27037EF3BF39C00886805D2704445AE7
:10E7B00020F9B1C43A240244443643948A9701971D
:10E7C0008A32940320C2BDE66A96522A06CC000D16
:10E7D0007EF01FCC0000DD46DD48DD4EDD50DD4C17
:10E7E000CC4000DD4A860F975ADC48D350DD58DC18
:10E7F00046D94F994EDD56DC58D34CDD58DC56D9FE
:10E800004B994ADD5674004E76004F7600507600E4
:10E8100051DC529356251E2606DC5493582516DCEF
:10E8200056DD46DC58DD48DC50D34CDD50DC4ED99B
:10E830004B994ADD4E74004A76004B76004C7600C8
:10E840004D74004A76004B76004C76004D7D005AA0
:10E850002609DC4EDD52DC50DD54397A005A20891D
:10E86000BDE66ADC522706CC000E7EF01F3CDC546D
:10E87000040453D74E16584FC3E8A218EC02DD46E5
:10E88000EC0093469748964E3D97499648D64E3DA4
:10E89000DB498900D346DD542A067A00527A0053B8
:10E8A000383940D840D835482E8629F4268423C8E4
:10E8B000217A1F7C1DC41C341AD6198C1856173E99
:10E8C000163A1540145A137412A211D01108104AA6
:10E8D0000F960EE20E2E0D840CDA0C3A0B9A0AFA01
:10E8E0000A5A09C40924088E07EE075806C2062CE6
:10E8F000058C04F6045603C00320028001D6012CC7
:10E900000082FFD8FF1AFE5CFD9EFCCCFBF0FB0AE8
:10E91000FA10F90CF7E0F6A0F524F376F15AEE8040
:10E92000EA20EA20BDE66A3C7D00522A09DC545305
:10E9300043C38001DD54DC54847FDD52188C4000D9
:10E94000182505CC80009352DD46164F05C3E9F922
:10E9500018EC00DD48EC02A300974E96473D975116
:10E960007F0050D64E96473DD350D3487F00527F0C
:10E9700000537D00542A154353730052730053C350
:10E98000000118DC52C9008900DD5218DD54383905
:10E99000BDE66A3C7F00567D00522A06BDF0867AAD
:10E9A0000056DC52270738CC000F7EF01FDC5427BE
:10E9B000462BF3CEE9F97F0057EC00189C5418243D
:10E9C0000708087C005720F1DD4A0909EC00DD4CFE
:10E9D000DC4A934CDD48CE0000DF46DC54934CDD2E
:10E9E000537F0055BDF17F96574A5FD354DD547D68
:10E9F00000562703BDF08638390000032406480975
:10EA00006A0C8C0FAB12C815E218F91C0B1F1A22E6
:10EA100023252828262B1F2E1030FB33DE36BA394B
:10EA20008C3C563F1741CE447A471C49B44C3F4E6C
:10EA3000BF5133539A55F558425A825CB35ED76042
:10EA4000EB62F164E866CF68A66A6D6C236DC96FEE
:10EA50005E70E2725473B575047641776B78847991
:10EA6000897A7C7B5C7C297CE37D897E1D7E9C7F12
:10EA7000097F617FA67FD87FF57FFFCC0002DD5440
:10EA80005FDD5239CC00E0DD547F00527F00533906
:10EA9000CC000020F2CC00107EF01FBDE66ADC52F4
:10EAA00026F3965426EFD655BDF09E5D27E7C1218B
:10EAB00024E386BF948A9701978A968B8A14978B52
:10EAC000972071EB157210152012780055790054BB
:10EAD00079005379005272041571FB157B400327AE
:10EAE000037C00555A26E339CC00117EF01FBDE6A9
:10EAF0006ADC5226F3DC5427403C18968A84FE9741
:10EB000001978A867EB70109CCEB3AFD010A7F00A6
:10EB1000547F005596431A914327FB01010101D60A
:10EB200008DC0D9643C6120FD7080E1A914327F73B
:10EB300096430926F27F00083839960884EF970833
:10EB4000DC0DDC54C30001DD54DC52C9008900DD5A
:10EB5000523B9608DE4A08DF4A84E29708DE0DDF62
:10EB600054B4C42B270EDE548C80002407DE5208D8
:10EB7000DF52DC093B960820F47EF3BFCC00127E06
:10EB8000F01F8628BDEEFB26F0BDE41EDC5226EC0D
:10EB9000DC5427E8183C18862CBDEEFB26DBBDE4D0
:10EBA0001EDC5226D7DC5427D3DD4E183818DD5032
:10EBB0008629BDEEFB26C23C968A84FE9701978A81
:10EBC000867EB70109CCEB52FD010A867EB70103B0
:10EBD000CCEB75FD01047F004A7F004B7F004CC6E3
:10EBE00002D708D608DC0DDC099643C6160FD708F5
:10EBF0000E1A914327099643DE4E092731DF4E0F47
:10EC0000DE4A092611964C260D7C004CDE52DF466A
:10EC1000DE54DF4820D79C5026D30E7F0008DC54FA
:10EC20009348DD54DC52D2479246DD5238397F009A
:10EC300008CC0000DD52DD543839BDE66A7F005A49
:10EC4000DC522A06CC00137EF01F3C2715740052BC
:10EC50007600537600547600557C005ADC5226ED3F
:10EC60002011DC5427DE2B0B7800557900547A00F4
:10EC70005A20EF7F00467F0047DC54C3B172DD4865
:10EC80007C0047CCB172DD52CC17ADDD54BDF17FB5
:10EC9000DC54DD567F0058DC4FDD52965197547F8F
:10ECA0000055BDF17FDC54D357DD57965689009748
:10ECB00056965680809756DC5805DD58DC565949E3
:10ECC000DD56730056DC574353C30001DD5796569B
:10ECD00089009756CE0000DC56DD54DD482A03CE6D
:10ECE000FFFFDF52DF46BDF25DDC4EDD5EDD54CC62
:10ECF000994BDD48CC0000DD46DD52BDF25DDC4EB7
:10ED0000C3F622DD54DC5EDD48CC0000DD52DD467A
:10ED1000BDF25DDC4EC3E2A8DD60CC0002DD5EDC4E
:10ED200057DD544FD6562A0286FFDD52DC54363763
:10ED300005DD58DC5236375949DD56CC0000DD463A
:10ED4000974896609749BDF25DDC4FD358DD58DC9B
:10ED500056C9008900DD564FD64E2A0286FFD3568B
:10ED6000DD56D661D7493332DD523332DD54BDF240
:10ED70005DDC4ED358DD58DC56C9008900DD564FA6
:10ED80005F7D004E2A03CCFFFFD356DD56DC578350
:10ED9000875DDD539656820097524F965A9B529745
:10EDA00052DC53DD5436374FD6522A0286FF3637AF
:10EDB000DD5286B19749CC0000DD469748BDF25D33
:10EDC000DC4EDD56DC50DD58C672D7493332DD5299
:10EDD0003332DD54BDF25DDC4ED357DD548600D6B0
:10EDE000562A0286FFC90089007D004E2A03C3FF10
:10EDF000FFDD523839BDE66ADC522B0B83000A2551
:10EE000006CC00147EF01FDC52DD56DC54DD58DCED
:10EE100053DD5496529753CC0001DD46CC62E4DDBD
:10EE200048BDF25DD64E2A0CC1F02408CC0000DDAE
:10EE300052DD54394F5CD75A2A0286FFDD5416DD65
:10EE400052CCB172DD487F00467F0047BDF25DDCE9
:10EE5000509358DD54DC4ED2579256DD52DC524767
:10EE600056DD5EDC544656DD608607975B3CCCFF82
:10EE7000FFDD52CCFFF3DD54CEEEDFBDEEAB7A000A
:10EE80005B26F8965A2B13270F7800557900547992
:10EE900000537900524A26F13839770052760053F0
:10EEA0007600547600554C26F13839DC5EDD46DCC0
:10EEB00060DD48BDF25D965048DC4E5949DD54CCCA
:10EEC00000007D004E2A03CCFFFFDD52EC02D3543C
:10EED000DD54EC00D9539952DD5208080808390076
:10EEE00000005BFFFFFDDE00000AABFFFFD5550011
:10EEF000008000FFFF000000010000160908A600C6
:10EF0000812027F908112701093908A60081202747
:10EF1000F939BDF39A7EF3BF0908A600812027F9CD
:10EF2000813F262608A600812027F981282705CCC5
:10EF300000400C39BDE66ADC522627DC544D2622FF
:10EF4000C106241E0505C373B0398040240139264B
:10EF50002008BDE66ADC522609DC5418BC72881809
:10EF60002506CC00027EF01F05054353C372190C21
:10EF700039811B25020D39084848164FC3721839CC
:10EF8000BDF09E7F0044BDEF0B7F00468126260327
:10EF90007EF0408130240139813A250139840F7D8A
:10EFA0000044260A7C0044975508A60020E57C0012
:10EFB00044D644C10524149747DC5405DD540505A7
:10EFC000D354D346DD5408A60020C89747DC540527
:10EFD000DD54DD50DC5259492B42DD52DD4E7800C4
:10EFE0005179005079004F79004E2B3078005179DB
:10EFF000005079004F79004E2B22DC54D350DD5461
:10F00000DC52D94F994E2B14DD52DC54D346DD54DB
:10F01000DC52C90089002B04DD5220AACC00033C3D
:10F02000CEF0267EF3C5484F573F20204552524F21
:10F0300052202300574841543F0D534F5252590D0F
:10F0400008A600814827090939964426020909398A
:10F0500008A600803025F2810A250A8007810A254A
:10F06000E8811024E47C0044D644C10924AEC604DF
:10F070007800557900547900537900525A26F19B53
:10F080005597557EF050730052730053DC54435330
:10F09000C30001DD54DC52C9008900DD52397F0014
:10F0A000527F00537F00547F0055393CFE738C3CE7
:10F0B000CEF0D3FF738CBDF0E938FF738C38393C48
:10F0C000FE738C3CCEF0D3FF738CBDF14438FF73DC
:10F0D0008C38390001004441544146494C45204F89
:10F0E00056455252414E4745003CBDF0EF38393647
:10F0F0007D00642609DC65052504811F2506CC00FA
:10F10000047EF01F331807360F18D7BC4C1684073F
:10F11000585858C4C0DA15D7159A179717DC668463
:10F120007FC340001896BCA70071F817713F1516F1
:10F13000320637DC66C30001DD66DC64C900890085
:10F14000DD6432393CBDF14A38397D00642609DC82
:10F1500065052504811F2506CC00057EF01F1607D6
:10F16000365C170F8407585858C4C0DA15D7159A5B
:10F17000179717DC66847FC3400018A60020AADE1C
:10F1800046264BDE4826083838CC00067EF01FDEC7
:10F1900052263BDC54CE00007C00527800497900B6
:10F1A0004824F576004876004993482404D3482043
:10F1B00001087A0052270B18051874004876004998
:10F1C00020E7DF54CE0000DF52DF4EDD50397F00F4
:10F1D0004ADE52DF4EDE54DF50CE0000DF52DF54F5
:10F1E0007C004A7800497900487900477900462434
:10F1F000EF760046760047760048760049DC50936B
:10F2000048DD50DC4ED2479246DD4E2410DC50D310
:10F2100048DD50DC4ED9479946DD4E20127C005522
:10F22000240D7C005424087C005324037C00527A73
:10F23000004A271A78005579005479005379005212
:10F2400074004676004776004876004920AF393C86
:10F25000CE004686106F00084A24FA38397F0044F1
:10F260007D00522A067C0044BDF0867D00462A1AA5
:10F270007A0044730046730047DC484353C30001DF
:10F28000DD48DC46C9008900DD46BDF2B3964E2A52
:10F2900006CC00077EF01F9644271773004E7300BC
:10F2A0004FDC504353C30001DD50DC4EC9008900E0
:10F2B000DD4E397F004E7F004F9649D6553DDD50DB
:10F2C000D655272F9648270B3DD34FDD4F964E89B5
:10F2D00000974ED6559647270A3DD34EDD4E240360
:10F2E0007EF371D6559646270A3D4D26F3DB4E2513
:10F2F000EFD74ED65427389649270B3DD34FDD4FD5
:10F30000964E8900974ED654964827083D4DD34EC9
:10F3100025CEDD4EF6C42FC1452614D65496472778
:10F320000A3D4D26BBDB4E25B7D74E964626B1D6B5
:10F33000532723964927093DD34EDD4E2533974E5B
:10F34000D6539648270A3D4D2627DB4E2523D74E18
:10F3500096479A46261BD65227169649270A3D4DB0
:10F36000260FDB4E250BD74E96489A479A46260124
:10F3700039CC00077EF01FBDEF1825433736863D98
:10F38000BDEEFB263ABDE41EDF46380FDC52ED0031
:10F39000DC54ED020EDF52DE4639863ABDEEFB2626
:10F3A0000532327ECB14860DBDEEFB2606323208C6
:10F3B0007ECADE39BDEF0B810D27F8813A27F43C78
:10F3C0004F5FCEF0340EDD547F00527F0053CCFBF4
:10F3D000A3DDAC7F00B57D008127273CFE738C8CBC
:10F3E000FFFF38271D96B681182606BDFBA37F00B8
:10F3F000B68EBFFFCC0000FD738EFD7394DE82BD20
:10F40000CAEC7F00B37F00B496B6270CBDFBA39671
:10F41000B6811826037F00B64FBDF55D860AB7B5E5
:10F420009ADC5427097F0045BDF598BDF6DCFE73D4
:10F430008C8CFFFF26037ECDF4EC0026037EC706EE
:10F44000BDF632183809DF4618A600810D270FBD1A
:10F45000F6DE9C462605863FBDF6DE0820EBBDF6AF
:10F46000DE7EC7063CCEF03A4F5F7EF3C5C60DD7B1
:10F470004636DF5218C300F0DD54DE52BDFB668114
:10F480007F27418108273D810A27F1810027ED81EF
:10F490000326113337C13A260B33383838FF738CC3
:10F4A000387EF6FFA700089146261233C13A270C92
:10F4B000BDFBA3810D2605860ABDFBA339BDFBA3B9
:10F4C0009C5426B89C5227B4098608BDFBA386200D
:10F4D000BDFBA38608BDFBA320A2DE548C800025C3
:10F4E00008CC00087EF01F3232CE73D2BC73A22546
:10F4F000040D86FF39EC00847F9354250139E60220
:10F50000DF564FD3561820E4200108A6002AFB201E
:10F51000DB3CDE52270738CC00087EF01FDE548C1F
:10F52000800024F2FE738CEC00847F26035D27B7F5
:10F53000189C543825D2FE738C200C09E6000886EE
:10F54000FF50DF56D35618DC548A80A1002605E10F
:10F55000012601398C73D226E20D86FF3916A600EA
:10F5600008112601393637BDF6DE3332810D26EE1D
:10F57000398622BDEEFB260ABDF55D810D26010907
:10F580004F398627BDEEFB27EF817F260A810826AB
:10F5900006860D9DAB20E9393C964536848097441C
:10F5A0009645847F97458614367A0045F6B59AC10C
:10F5B0000A260E7D00522A09BDF0867C00447A009E
:10F5C00045F6B59A4F18DF487F00477F0046BDF1EA
:10F5D0007FDE522604DE542708D651377A004520B4
:10F5E000E0D651377B804427159644840127048652
:10F5F0002D9DAB7A00452B1B86309DAB20F57A0004
:10F60000452B0686209DAB20F59644840127048671
:10F610002D9DAB328114270C810A25028B078B307C
:10F620009DAB20EF3297453839BDF6324FBDF55DC1
:10F630000839EC00847FDD547F00527F00530808B6
:10F640000886049745BDF5988620BDF6DE39FE7321
:10F65000A4BC73A8260139A600083CFE73A6A70027
:10F6600008FF73A63820EAFE73AABC73AE260139E0
:10F6700009A6003CFE73AC09A700FF73AC3820EA72
:10F680003233DF5E38FF7394271838FF739A38FFE0
:10F69000739C38FF739638FF739838FF739E38FF5A
:10F6A00073A03736DE5E393233DF5E308CB601242C
:10F6B00005DE5E7EF464FE7394271BFE73A03CFEA1
:10F6C000739E3CFE73983CFE73963CFE739C3CFE1E
:10F6D000739A3CFE73943C3736DE5E39860D369D58
:10F6E000AB3236810D2604860A9DAB32397D0093FC
:10F6F0002601397D009E27FA7F0093BDFB040E7D15
:10F70000008C271A8EBFFDCC0000FD738EFD739414
:10F71000CC0064DD54CC0000DD523C7ECB23FE7374
:10F720008C2727CEF74DBDF6DC4FBDF55DFE738C03
:10F73000EC00847FDD547F00527F00537F004586BC
:10F740000AB7B59ABDF598BDF6DC7EC706425245AC
:10F75000414B204154204C494E4520000F36BDF806
:10F760003932843F8A8016BDF78871DF17BDF803F0
:10F77000D756BDF803D757BDF84A0E200439BDF758
:10F780008871DF1771BF173971DF1771BF1771EFFC
:10F790001772401772201771DF1772101772201737
:10F7A0008608BDF826390F3632843F36C630BDF79D
:10F7B0007E32368AC016BDF788BDF7DD0E01010F17
:10F7C00032843F8A4016BDF788D656BDF824D657F6
:10F7D000BDF824BDF7DDC600BDF77E0E3971EF1709
:10F7E00071DF1771BF17CE04C47220170101010128
:10F7F00071DF170926F372401772201771DF177136
:10F80000BF1739C60272201771DF177B081727014F
:10F810005C7220175824F171DF177B081727015CF1
:10F820007220173986085871DF1772101725037177
:10F83000EF177220174A26EE399617844797178AD2
:10F8400040971739BDF839BDF8797B02BB271E7B7D
:10F8500004BB271E3C18C601BDF91C72201771DFBE
:10F860001772201771DF177240171838397B04BBE5
:10F870002606718717728017390F3C189617168461
:10F88000CF971784BF97177B02BB27037EF8FA1820
:10F8900053CB088604C1082505721017200371EFA9
:10F8A0001772201771DF1758C40F4A26E8961716EB
:10F8B000CA20D7179717D7179717D7179717D7179C
:10F8C0009717D7179717D717BDF956CE0004090118
:10F8D0000101010126F8CE000A4F5F057B081727BA
:10F8E00002CB4072201771DF170926EF72401738DC
:10F8F0000E39F4B4E4A4D494C484184FC3F8F218B5
:10F90000D6BBC408EA00BDF91C86104A26FD860253
:10F91000BDF9333686104A26FD3220D38608582496
:10F9200005721017200371EF1772201771DF174A45
:10F9300026EC39CE000C5F052405721017200371E8
:10F94000EF177B081727015C72201771DF17092654
:10F95000E60505050539CE00050926FD97173996F8
:10F960001784CF971784BF9717D6BBC408FAF8F24D
:10F97000BDF91C3686104A26FD320F3C7C0053D65A
:10F98000534FC3F8F21896BB8408AA008A02BDF947
:10F99000330E38BDFA26D653D15226DE7EF84F9765
:10F9A00052D7467F0053BDF8397B02BB27037EF94F
:10F9B0005F0F3C71EF1771BF1772201771DF17725D
:10F9C0001017CE000972201771DF170926F7CE0035
:10F9D0000309010101010126F87C00539653438B72
:10F9E000089754CE000A4F5F71DF177800547B10E0
:10F9F000542705721017200371EF17057B0817278E
:10FA0000015C7220170926E071DF170E3805050525
:10FA1000050505BDFA269652915327043C7EF9CE82
:10FA20007240177EF86D7D004627167A004626053F
:10FA30007C004620087C004637BDF0E932BDF0E985
:10FA40003905057B02BB27F5050520F1961E84D0FC
:10FA500027558450270396123BDE719612A7007B30
:10FA60000176271281132605728076203A811126AD
:10FA700005717F762031810326037C0093098C7207
:10FA80008B2603CE738BDF717D0075261A18937356
:10FA9000C1402613FCB596B3B594C1FF2709861360
:10FAA000BDFBA386FF977596118424812427013B13
:10FAB0007B017627237B8076271EDEAFBDF6ED71B6
:10FAC000FB110E010196431A914327F90F092705EF
:10FAD0007B807626E7717F76FEB596A600098CB40A
:10FAE000932603CEB593FFB5967D00772602971334
:10FAF000FEB596BCB594260471FB113B7204113B14
:10FB000086FF97753CCE738BDF71DF7371FB11CE6F
:10FB1000B593FFB594FFB596967527088611BDFB82
:10FB2000A37F007538717F767F0093399674907249
:10FB300039B6B597B0B59539DE643CDE663CDEB3C8
:10FB4000EC00DD64EC02DD663CBDF14438D664E7D0
:10FB500000D665E701D666E702D667E70338DF66B9
:10FB600038DF643338393C3736DCB33226CADE73CB
:10FB70009C7126031A20F7A60036098C728B260387
:10FB8000CE738BDF739675270F189371C1402608CB
:10FB90008611BDFBA37F0075323338810326037ABB
:10FBA0000093393C3736FCB596B3B594C1FF27F6C0
:10FBB000FEB59432A700098CB4932603CEB593FF0B
:10FBC000B59472041133383986209DAB86209DABE5
:10FBD00039DE6C08DF6C7A00B82619DC42C30001FC
:10FBE000DD42DC40C9008900DD4096AE890097AE59
:10FBF00096B797B8717F1B3B3B3B8E00FD86029703
:10FC000090BDFC141A1A1ACE0000DF42DF407F00BC
:10FC1000AE7EC68B8612971B7F00017F008A86C04E
:10FC20009720978B7F0015860A9711860597108677
:10FC3000E097148640971786F797169770860B976C
:10FC4000BBBDF84486029790860397707F0091862B
:10FC5000FF9780867EB7010FCCFBD1FD0110865F38
:10FC60007B01BB270286BF971C9763860197B897D5
:10FC7000B772401B0E86FF9777392A202050433DEC
:10FC80002420413D2420423D2420463D2420583D4F
:10FC9000242040583D242053503D24204024DEACF5
:10FCA0003CCEFBA3DFAC0E860DBDFBA3860ABDFBDD
:10FCB000A3CEFC7ABDFD363C30EC091809BDFD3EF3
:10FCC00038BDFD363C30A606BDFD4338BDFD363C93
:10FCD00030A605BDFD4338BDFD363C30A604BDFD54
:10FCE0004338BDFD363C30EC0718BDFD3E38BDFD48
:10FCF000363C30EC0718EC0018BDFD3E38BDFD3633
:10FD00003C3018C3000A18BDFD3E38BDFD36FE72FA
:10FD100082BDFD3E863DBDFBA3FE7282860836A6EF
:10FD20000008BDFD438620BDFBA3324A26F038DF24
:10FD3000AC3BBDFBA308A600812426F608393C3263
:10FD40008D013236444444448D0132840F8B30811E
:08FD50003A25028B077EFBA39C
:10FFC7007EFB317EF8797EF8397EF84A7EF0AB7E8B
:10FFD700F0BF7EFB2C7EFB667EFBA37EFB047EF8D8
:10FFE7004400DF0100010FFBF8FA4C010301060191
:09FFF70009010CFC9EFBF9FBFA68
:00000001FF
